:100000000C941E010C9456010C9456010C9456014C
:100010000C9456010C9456010C9456010C94560104
:100020000C9456010C9456010C94661C0C94381DCB
:100030000C945A170C9456010C9456010C945601CA
:100040000C9456010C9456010C9456010C945601D4
:100050000C9456010C94E2170C9456010C94560122
:100060000C9456010C9456010C9456010C945601B4
:100070000C9456010C9456010C9456010C945601A4
:100080000C9456010C9456010C9456010C94560194
:100090000C9456010C9456010C9456010C94560184
:1000A0000C9456010C9456010C9456010604060457
:1000B000320432049A04B804D005D005C3045C05A8
:1000C0006D056D05A51DCC1DC41ECC1DC41E181EBE
:1000D0003B1EC41E921EA11E040005000600070060
:1000E000080009000A000B000C000D000E000F00B4
:1000F0000000100011001E03770061007A006F00FD
:10010000770073006B0069002000320033002D007F
:1001100031003900000018036B00650065006200C3
:100120007A0064006F0074006E00650074000000C7
:100130000403090409023B00020100A0FA090400BB
:100140000001030101000921110100012240000703
:1001500005810308000109040100010300000009F2
:100160002111010001227B000705820320000112FA
:10017000010002000000085A4BFC5301000102007C
:100180000105010902A10185020901A10005091962
:10019000012908150025019508750181020501094D
:1001A0003009311581257F950275088106093815BA
:1001B00081257F950175088106050C0A3802158195
:1001C000257F950175088106C0C005010980A10140
:1001D000850319012AB700150126B700950175108E
:1001E0008100C0050C0901A101850419012AA002A2
:1001F000150126A002950175108100C005010906B0
:10020000A101050719E029E71500250195087501E9
:1002100081029501750881010507190029FF150064
:1002200026FF009506750881000508190129059526
:100230000575019102950175039101C011241FBE3E
:10024000CFEFDAE0DEBFCDBF04B603FE18C0809169
:10025000340290913502A0913602B0913702873076
:10026000904BA740B04B59F41092340210923502D3
:100270001092360210923702E0E0F8E3099511E09F
:10028000A0E0B1E0EEEEFEE302C005900D92A438CE
:10029000B107D9F722E0A4E8B1E001C01D92A43370
:1002A000B207E1F70E94A4110C94751F0C94000092
:1002B00081E0089581E008950C945A0108950C940A
:1002C0005E011F93CF93DF9300D000D01F92CDB774
:1002D000DEB749835A836B833091870189819A8184
:1002E000311114C0662359F0222349F00E940F08EF
:1002F000182F682F89819A810E94B60703C00E9437
:10030000E207182F69817A81812F04C00E940F08AB
:1003100069817A810F900F900F900F900F90DF916D
:10032000CF911F910C94300FFC01262F40815181F9
:100330006281738184810C94610181E00895CF937F
:10034000DF93EC0160E00E949401BE01DF91CF9148
:100350000C945F010C9473100C946F1008950E941C
:1003600060060E94AE012FEF84E39CE021508040A4
:100370009040E1F700C000000C9408180F931F9301
:10038000CF93DF938C0161E00E949401EC01B801EE
:100390000E945C018823F1F1B801CE010E9426166B
:1003A0008823C1F1B801CE010E943A14882391F14B
:1003B000B801CE010E948215882361F1F801828183
:1003C000882309F1CB358DE5D807C1F050F4C1156C
:1003D000FCE5DF0781F0CF3DDC45A9F40E94460D26
:1003E00019C0CC35EDE5DE0761F0CD35DD4559F4BA
:1003F0000E94890C08C00E94AF010CC00E94920CA0
:1004000002C00E94950CC801DF91CF911F910F91FE
:100410000C94580180E0DF91CF911F910F910895C6
:100420000E943D170C9429020E942C020C94431741
:1004300008950C94180281E008950C941B0208950D
:10044000CF93C82F0E9419028C2F0E941D02CF91BA
:10045000089580E00C9420020E9482160C942002E1
:100460000E94821690918601891721F0809386015F
:100470000C9420020895CF93DF93CDB7DEB72B976E
:100480000FB6F894DEBF0FBECDBF4F835887698784
:100490007A878B8761110E94D50B9E012F5F3F4F9A
:1004A00086E0F90111928A95E9F785E0FE01379619
:1004B000D90101900D928A95E1F789819A814C8149
:1004C0005D81452B31F09F3F31F491E08F3F19F46E
:1004D00003C091E001C090E090FF09C049815A81BA
:1004E0006B817C818D819E810E94F60A05C0C901C5
:1004F0000E949D018111F2CF2B960FB6F894DEBFBA
:100500000FBECDBFDF91CF910895FC018081918115
:100510000E9451080895CF93882309F4A4C0C82FDE
:100520008238C1F40E94821681FD9DC069E38091EA
:100530000201909103010E9415170E94F70B2FEF03
:1005400081EE94E0215080409040E1F700C000002F
:1005500069E319C0833801F50E94821680FD83C0CB
:1005600063E580910201909103010E9415170E949A
:10057000F70B2FEF81EE94E0215080409040E1F79F
:1005800000C0000063E580910201909103010E9488
:100590001717CF910C94F70B8438C1F40E94821680
:1005A00082FD61C067E480910201909103010E9485
:1005B00015170E94F70B2FEF81EE94E02150804039
:1005C0009040E1F700C0000067E4DDCF8CEF8C0FB6
:1005D000813AD0F46C2F80910201909103010E9426
:1005E000DF16882349F06C2F80910201909103015E
:1005F0000E9417170E94F70B6C2F809102019091B7
:1006000003010E941517C5CF80E28C0F883048F493
:10061000C77081E001C0880FCA95EAF70E94B80B45
:10062000B8CFEBE5EC0FE33040F4F0E0E95BFE4FD0
:10063000808190E0CF910C94A716E8E5EC0FE731AC
:1006400050F4F0E0EE0FFF1FE75EFE4F80819181D6
:10065000CF910C94BD16CD3E30F08C2F0E94291204
:10066000CF910C94FB12CF910895882309F464C0B4
:10067000823879F40E94821681FF5EC069E380911E
:100680000201909103010E9415170E94F70B69E384
:1006900010C08338B1F40E94821680FF4DC063E51C
:1006A00080910201909103010E9415170E94F70B9F
:1006B00063E580910201909103010E9417170C9449
:1006C000F70B843879F40E94821682FF35C067E404
:1006D00080910201909103010E9415170E94F70B6F
:1006E00067E4E7CF9CEF980F913A10F4682FE1CFC1
:1006F00090E2980F983050F4877091E001C0990F04
:100700008A95EAF7892F0E94BE0BD9CF9BE5980FF7
:10071000933020F480E090E00C94A71698E5980FB1
:10072000973120F480E090E00C94BD168D3E20F0CF
:100730000E9484120C94FB1208951F93CF93DF93B1
:10074000182FEB010E948B02209741F08FE99FE068
:100750000197F1F700C000002197F6CF812FDF91BC
:10076000CF911F910C943503893319F060E070E04C
:1007700002C060E570E00C949D03882321F00E9484
:10078000B80B0C94F70B0895882321F00E94BE0B40
:100790000C94F70B0895CF92DF92EF92FF920F9394
:1007A0001F93CF93DF937C01D62FC72FFC011281BB
:1007B000058102950F700E94AE0B8823B9F01123BA
:1007C000A9F08C2F807F803421F080E28D0F88305B
:1007D00068F080911C0282FD09C082E00E94570CE3
:1007E0000E94AE0B91E0D82ED92601C0D12CCC2E80
:1007F000C2948FE0C8228C2D90E08C30910508F0D7
:10080000CFC1FC01EA5AFF4F0C940C1F8C2F807F44
:10081000CF70882311F0C295C07F112399F0CC23AB
:1008200009F4AAC180E28D0F883010F0D11104C004
:100830008C2F0E94B80B03C08C2F0E94C80B0E9403
:10084000F70B9AC18D2F0E943503CC2309F4A8C160
:1008500080E28D0F883038F1DD2329F18C2F0E9442
:10086000CE0B24C08C2F807FCF70803211F0C295C8
:10087000C07FDD2319F0D130A1F13DC080911C0271
:1008800082FF17C0112349F0CC2329F08C2F0E943E
:10089000B80B0E94F70B80E070C180E00E94350326
:1008A000CC2309F47DC18C2F0E94BE0B0E94F70B54
:1008B00077C1112371F0002341F0013031F40E941F
:1008C000D80B8C2B0E94E00B6BC10E94D80B8C2B99
:1008D0001DC0002319F0013009F462C10E94ED0B24
:1008E00025C0112321F0063008F05AC10EC0053092
:1008F00008F056C11BC0112361F0002331F0F7014D
:10090000858180FF39C18F7085838C2F0E94BD0344
:1009100047C1002359F0D93309F03FC1FFEF07EE7B
:1009200013E0F15000401040E1F735C18C2F0E94D8
:10093000C40336C18C2F86958695837019F081305B
:1009400061F02EC1112321F08D2F9C2F937002C0D6
:1009500080E090E00E94A7162BC1112321F08D2F7B
:100960009C2F937002C080E090E00E94BD1620C1D1
:100970008D2F112319F00E94291202C00E948412A7
:100980000E94FB1215C18C2F837009F047C0111112
:100990000BC12D2F229526952770220F220F6D2F28
:1009A0006F70862F90E0A0E0B0E0022E04C0880FA8
:1009B000991FAA1FBB1F0A94D2F7D4FF10C04FE0A3
:1009C00050E060E070E004C0440F551F661F771FC1
:1009D0002A95D2F7409550956095709503C040E0F8
:1009E00050E0BA01C695C695C3708A019B01082BD9
:1009F000192B2A2B3B2BC901B801C23049F058F4FE
:100A0000C13019F00E94CC06CFC00E94BA06CCC0FB
:100A10000E94DE06C9C00E94B806C6C0112319F0A4
:100A20008C2F817001C08695882309F4BDC02D2FBD
:100A3000229526952770220F220F6D2F6F70862F1B
:100A400090E0A0E0B0E0022E04C0880F991FAA1F1A
:100A5000BB1F0A94D2F7D4FF10C04FE050E060E013
:100A600070E004C0440F551F661F771F2A95D2F708
:100A7000409550956095709503C040E050E0BA01F4
:100A8000C695C695C3708A019B01082B192B2A2B8A
:100A90003B2BC901B801C23049F058F4C13019F0FC
:100AA0000E94910781C00E947F077EC00E94A30719
:100AB0007BC00E94F20678C0CF70112339F08C2FD2
:100AC0000E9418078D2F0E94BD036EC08D2F0E94BB
:100AD000C4038C2F0E94390767C0D23F21F128F44C
:100AE000D03F41F0D13FC1F043C0D33F19F1D43FD3
:100AF00079F03EC0112341F0053008F051C08C2F31
:100B00008F710E945E074CC0063008F049C0F7CFD5
:100B100080911C0282FF18C0112339F08C2F8F7135
:100B20000E9418073DC01123C9F38C2F8F710E94BA
:100B3000390736C0112329F08C2F8F710E940307CB
:100B40002FC00E94FE062CC0112349F0CF718C2FBC
:100B50000E94180763E08C2F0E943C0C21C081E0AA
:100B60000E94570C0230E0F082E00E94570C18C03F
:100B7000112331F0002391F28D2F0E948B0210C0BF
:100B8000002399F2D93349F41FEF27EE33E01150D7
:100B900020403040E1F700C000008D2F0E94350357
:100BA00088EF8C0D843020F40E9482160E9420026F
:100BB000DD20C9F00E94AA0B80FD15C0F70112824A
:100BC0000E94A40B0E941807C7010E9414060E94ED
:100BD000A40BDF91CF911F910F91FF90EF90DF90C9
:100BE000CF900C943907DF91CF911F910F91FF9017
:100BF000EF90DF90CF9008950F931F93CF93DF93E3
:100C0000EC01688179818A810E945C088C010E94D4
:100C1000B5070E94A606B801CE010E94CB03DF9162
:100C2000CF911F910F910895CF93DF93EC0198819D
:100C300089812B813C81232B31F08F3F31F481E07E
:100C40009F3F19F403C081E001C080E080FD1DC01A
:100C5000CE010E94BE01811110C00E94AE0B8823FC
:100C6000A1F08A81882389F080911C0282FD0DC049
:100C700082E0DF91CF910C94570CCE010E94FC05CD
:100C8000CE01DF91CF910C949F01DF91CF91089518
:100C900080E090E00E94A71680E090E00E94BD16E0
:100CA0000E94D50B0E94F70B0E942C140C94FB128F
:100CB00080910201909103010E9419170C9448063B
:100CC0000E94C50B0C94580692959F70963079F04F
:100CD00010F4925001C09A50923068F4803F69F04D
:100CE00018F4883E40F409C0843F29F406C0883EC9
:100CF00020F0813F11F080E0089581E00895FC012B
:100D0000808191810E9451080E9464060895CF93CA
:100D1000DF9300D000D01F92CDB7DEB70F900F90B9
:100D20000F900F900F90DF91CF910895CF93DF93A5
:100D300000D000D000D0CDB7DEB726960FB6F8941D
:100D4000DEBF0FBECDBFDF91CF9108950895089506
:100D50000C94A7060C94A8060E94AA06609396011C
:100D60007093970180939801909399010C94480691
:100D70000C94AC060F931F9300919601109197016C
:100D80002091980130919901602B712B822B932B2C
:100D90001F910F910C94AC060F931F930091960135
:100DA000109197012091980130919901602371234E
:100DB000822393231F910F910C94AC060F931F93E2
:100DC000009196011091970120919801309199011D
:100DD00060277127822793271F910F910C94AC06EF
:100DE0000C94A7060E94F006609392017093930101
:100DF00080939401909395010C94480660E070E014
:100E0000CB010C94F2060F931F9341E050E060E099
:100E100070E08A019B0104C0000F111F221F331FC5
:100E20008A95D2F7C901B8011F910F910C94F2066F
:100E30000F931F9341E050E060E070E004C0440F66
:100E4000551F661F771F8A95D2F780919201909166
:100E50009301A0919401B09195018A019B01082B07
:100E6000192B2A2B3B2BC901B8011F910F910C9410
:100E7000F2060F931F9341E050E060E070E004C081
:100E8000440F551F661F771F8A95D2F740955095DE
:100E9000609570958091920190919301A091940139
:100EA000B09195018A019B01082319232A233B2332
:100EB000C901B8011F910F910C94F2060F931F9373
:100EC00041E050E060E070E004C0440F551F661F31
:100ED000771F8A95D2F78091920190919301A0910A
:100EE0009401B09195018A019B01082719272A27AF
:100EF0003B27C901B8011F910F910C94F2060F9383
:100F00001F930091920110919301209194013091CF
:100F10009501602B712B822B932B1F910F910C94B9
:100F2000F2060F931F93009192011091930120916B
:100F300094013091950160237123822393231F91A3
:100F40000F910C94F2060F931F9300919201109150
:100F50009301209194013091950160277127822798
:100F600093271F910F910C94F206089524E0929F0D
:100F7000900D1124890FE82FE695E695E695877088
:100F800051E001C0550F8A95EAF785E0E89FF0012E
:100F90001124E857FE4F20E030E070E04081CB01A3
:100FA000022E02C0969587950A94E2F7817081958A
:100FB00084278523842781932F5F3F4F2530310578
:100FC00069F7089524E0929F900D1124890F682FEE
:100FD000669566956695982F977085E0689FB00135
:100FE000112440E050E080E0FB01E40FF51FE857DA
:100FF000FE4F208130E0092E02C0369527950A94D5
:10100000E2F721703327042E01C0220F0A94EAF779
:10101000822B4F5F5F4F4530510531F70895BF92E6
:10102000CF92DF92EF92FF920F931F93CF93DF93B4
:101030008C01C0909201D0909301E0909401F090C7
:1010400095018091960190919701A0919801B0919E
:101050009901C82AD92AEA2AFB2ACFE1D0E0D70190
:10106000C6010C2E04C0B695A795979587950A944E
:10107000D2F780FD04C0219790F7B12C07C0BC2E99
:10108000B8018C2F0E94430F0197A9F38B2DDF919C
:10109000CF911F910F91FF90EF90DF90CF90BF9075
:1010A0000895CF93DF93EC010E940F08BE010E94C8
:1010B000430FDF91CF9108951F93CF93DF93EB01FF
:1010C00090918701992321F0CB010E94510813C010
:1010D000882349F0CB010E940F08182F682FCE01FA
:1010E0000E94B60704C0CB010E94E207182FBE0180
:1010F000812F0E94430FDF91CF911F9108951F937D
:10110000CF93DF93C0919A0116E080919B01C8179D
:1011100099F0D0E01C9FF0011D9FF00D1124E456C2
:10112000FE4F4081518162817381848195810E944B
:1011300096062196C770E9CFDF91CF911F91089550
:101140004091CC015091CD016091CE017091CF01C1
:101150008091D0019091D1010C949606EF92FF926C
:101160000F931F93CF93DF938091D10182958F705E
:1011700009F065C08091CE01882309F460C0809198
:101180009A01F0909B011091CC010091CD016091EA
:10119000CF017091D00191E01F3F09F090E0C09124
:1011A0000001D0910101292F96E0E92E8F1509F455
:1011B00046C06115710521F00F3F21F030E003C0FA
:1011C00031E001C0322F90E030FD36C0E89EF001E2
:1011D000E99EF00D1124DF01A456BE4F11963C91FB
:1011E0001197301329C03C91311326C012963C91BF
:1011F0001297311121C013964D915C911497461BA3
:10120000570B4C175D07C0F48091D1018F7080613E
:101210008093D101EF55FE4F80818F708061808374
:101220008CEC91E00E941406DF91CF911F910F91F9
:10123000FF90EF900C947F0801968770B7CFDF91F5
:10124000CF911F910F91FF90EF9008959F92AF92D1
:10125000BF92CF92DF92EF92FF920F931F93CF93A3
:10126000DF93CDB7DEB761970FB6F894DEBF0FBE40
:10127000CDBF8C0185E0F801DE011D9601900D9235
:101280008A95E1F7D8011296EC909091CC01E0910B
:10129000CD012091CF013091D0012115310531F0E0
:1012A000EF3F31F481E09F3F19F403C081E001C0BA
:1012B00080E0B82FB1709B2E80FD47C1D8014C91C2
:1012C00011965C9111971396AD90BC9014978CEC8D
:1012D000C82E81E0D82EF090CE01B501621B730BB1
:1012E0002091000130910101FF2009F4D9C08091C3
:1012F000D1016217730708F095C0282F207F09F0ED
:1013000052C05E1313C0491311C0FE2CE1100EC071
:101310008F7080618093D1010E94A008C6010E9455
:1013200014068091D101F80185834DC1AB2831F0BD
:101330005F3F31F481E04F3F19F403C081E001C009
:1013400080E080FD03C081E08E2502C080E090E057
:10135000F82FF170FF2E80FF1CC080919A01209120
:101360009B0136E0821709F40BC190E0389FF00131
:10137000399FF00D1124E456FE4F6181561306C0CB
:101380006081461303C06281E61203C00196877034
:10139000E9CFFE2CEE2009F416C18091D1018160C5
:1013A0008093D10154C05E1306C0491304C0E110FC
:1013B00002C0F80199C0C8010E947F06882361F12C
:1013C000EE2051F12091D101822F82958F7090E013
:1013D000029774F08091CC019091CD0198878F8312
:1013E0001986BB86AA862C87CE0107960E94140612
:1013F00086E0F801ACECB1E001900D928A95E1F73E
:101400000E94AE080E94A0080AC05E1711F1C80130
:101410000E947F0681112CC0C8010E941406FF247F
:10142000F394D1C0282F207F81F77A2DB98AA88A1A
:101430006E2D89890E9487068CEC91E00E9414062B
:1014400086E0D6011D928A95E9F70E94A008F12C4A
:10145000BAC04913DCCFE110DACFF8018583C801A7
:101460000E94140686E0D6011D928A95E9F7ABC06A
:10147000EE2091F22091D101822F82958F7090E021
:1014800002970CF4B5CF8091CC019091CD019A8355
:1014900089831B82BD82AC822E83CE010196A6CFAA
:1014A0006217730708F044C0FE2CEE2009F4B4CF95
:1014B0005E1330C049132EC02091D10120FD21C000
:1014C000822F82958F70482F50E041155105C9F049
:1014D000F80125834F30510541F08F5F982F929589
:1014E000907F822F8F70892B8583C8010E941406FC
:1014F00086E0F801ACECB1E001900D928A95E1F73D
:101500003CC086E0F801ACECB1E001900D928A9508
:10151000E1F759C0C8010E947F06811169CF80910F
:10152000D10181608093D101C8010E9414064BC093
:101530007A2DB98AA88A6E2D89890E94870686E04D
:10154000D6011D928A95E9F718C0EE2009F464CF00
:10155000C8010E947F06F82E882309F45DCF86E03B
:10156000F801ACECB1E001900D928A95E1F78CECBA
:1015700091E00E9485020E94AE080E94A00823C04C
:101580004D875E878D859E850E945108292F229563
:101590002F70223028F49F7039F0811105C00BC0E4
:1015A000243028F49F7049F4805E883020F0C80110
:1015B0000E9414069F2CF92C06C0D80115969C9108
:1015C000907F91F7F8CF8F2D61960FB6F894DEBF1C
:1015D0000FBECDBFDF91CF911F910F91FF90EF9084
:1015E000DF90CF90BF90AF909F9008951F93CF93BF
:1015F000DF93CDB7DEB72C970FB6F894DEBF0FBEE2
:10160000CDBF4F83588769877A878B879C87CE01A8
:1016100007960E9426098823D1F09F8188852A8514
:101620003B85232B31F08F3F31F481E09F3F19F44C
:1016300003C081E001C080E080FD47C04F81588534
:1016400069857A858B859C850E9496063EC086E0DA
:10165000FE013796DE01119601900D928A95E1F711
:10166000FF81E8856A857B856115710531F0EF3F63
:1016700031F481E0FF3F19F403C081E001C080E054
:1016800080FD23C020919B0130E0C9010196877045
:10169000992740919A0150E084179507F1F1F98359
:1016A000EA837D836C8396E0929FD001939FB00D77
:1016B0001124A456BE4FFE01319601900D929A95C9
:1016C000E1F780939B010E947F0816E080919A01C8
:1016D00090919B01891771F1189FC00111248456C4
:1016E0009E4F0E942609882329F1E0919A011E9FAE
:1016F000F0011124E456FE4F4081518162817381D3
:10170000848195810E94960680919A0190E00196CD
:101710008770992780939A01D9CF0E946006109212
:101720009B0110929A01ECECF1E086E0DF011D9242
:101730008A95E9F72C960FB6F894DEBF0FBECDBFA1
:10174000DF91CF911F9108958091DA01859585955C
:10175000859508958091DA01877008959091DA0156
:10176000977081E009F480E008958091E501089583
:101770009091E501892B8093E501089580959091E2
:10178000E50189238093E50108951092E50108950C
:101790009091E401892B8093E401089580959091C4
:1017A000E40189238093E40108951092E4010895EF
:1017B0008091DB01089508950C94DB0B0C94DC0BF5
:1017C00090911C0292FD08C09091DB01981721F0C6
:1017D0008093DB010C94DE0B08958091DB0188235C
:1017E00029F01092DB0180E00C94DE0B0895CF937A
:1017F000DF93E0910201F09103018091E501808384
:10180000E0910201F091030190818091E401892B24
:1018100080838091DB01882381F0E0910201F091C7
:1018200003019081892B80838091020190910301B3
:101830000E94D31681110E94ED0BC0910201D0913C
:10184000030148E050E062ED71E0CE010E94261FE6
:10185000892B69F088E0FE01A2EDB1E001900D92C4
:101860008A95E1F7CE01DF91CF910C948E16DF912E
:10187000CF9108950C94DB0B90911C0292FD10C047
:1018800098E0899F90011124262B2093DA010E9471
:1018900018078091DA018595859585950C943A0C09
:1018A0000C9418071092DA0180E00C943A0C209105
:1018B000DA01809582238093DA01982F977099F44A
:1018C00030E0482F082E000C550B2417350759F02F
:1018D00090911C0292FD07C08595859585950E9483
:1018E00039070C94520C089590911C0292FB222708
:1018F00020F9281769F080FB92F990931C028091DF
:101900001B0290911C020E94C20C82E00C94570CA6
:10191000089580911C0282FB882780F991E0892735
:101920000C94740C81E00C94740C80E00C94740C96
:101930006FEF7FEF80E090E00C945F1F80E090E01D
:101940000E943B1F21E0893E9E4F09F020E0822F3C
:10195000089582E090E00C94331F83E090E00C94B3
:10196000331FCF9384E090E00E94331FC82F82E2A0
:1019700090E00E94331F2C2F30E0A901582BCA01A0
:10198000CF910895CF93C92F682F84E090E00E94F3
:10199000411F6C2F82E290E0CF910C94411FAB016C
:1019A000BC018FE090E00C94531FAB01BC0183E1BC
:1019B00090E00C94531F60E070E0CB010C94D50CC8
:1019C00060E070E0CB010E94CF0C0C94DB0C69EE60
:1019D0007EEF80E090E00E945F1F60E082E090E098
:1019E0000E94411F60E083E090E00E94411F10923E
:1019F000960110929701109298011092990160E05F
:101A000084E090E00E94411F60E082E290E00E944A
:101A1000411F60E085E090E00E94411F60E086E0A9
:101A200090E00E94411F6FEF87E090E00E94411F0D
:101A300040E050E0BA0188E090E00E94531F60E06F
:101A40008DE090E00E94411F40E050E0BA0188E143
:101A500090E00E94531F60E087E190E00E94411FE8
:101A600040E050E0BA018CE190E00E94531F60E03A
:101A700070E080E290E00E945F1F40E050E0BA0119
:101A800088E190E00E94531F0C94E00C0C94E70C4A
:101A9000682F8EE090E00C94411F0E94C71760935E
:101AA000ED017093EE018093EF019093F00160934C
:101AB000E9017093EA018093EB019093EC010895A2
:101AC00085B7806885BF85B7806885BF089581E048
:101AD00008950C94670D08950C946B0D0C946B0D88
:101AE0000C946E0D0C946B0D0C94720D0C946B0D8C
:101AF0000E94600D8FE190E10E9478160E94760DA1
:101B00000C94740D0E946C0D0C946B0D0E94391096
:101B10000C941F020E94B2170E9409110E94860DA8
:101B20000C94700D8F929F92AF92BF92CF92DF92E2
:101B3000EF92FF920F931F93CF93DF93CDB7DEB752
:101B40002A970FB6F894DEBF0FBECDBF0E941E11BC
:101B5000982E81110E944D0D86EEA82E81E0B82EA0
:101B600000E010E0802E802F0E945D10D82EF5013D
:101B7000C1905F01C826B1F40F5F1F4F03301105FC
:101B800089F78FEF89838A831B820E94BB1781604C
:101B9000782F9D838C8349815A816B818D810E942E
:101BA0003B022FC08091F10181FD0E946310E12C66
:101BB000FF24F3948C2D8F21F1F00E94690D88236E
:101BC00099F0EE828F82DF2081E009F480E088873F
:101BD0000E94BB178160782F9A8789874E815F8129
:101BE00068858A850E943B02F801EA51FE4F808198
:101BF000F826F08206C0E394FF0CF5E0EF12DACF8E
:101C0000BBCF81E0911001C080E02A960FB6F89416
:101C1000DEBF0FBECDBFDF91CF911F910F91FF901F
:101C2000EF90DF90CF90BF90AF909F908F900895EE
:101C30000E94920D0E9419130C943002CF93DF93EF
:101C40000E94480FEC01811521E5920708F045C07C
:101C5000811530E5930708F094C0883E910528F57A
:101C6000803E910508F0F8C0883A910570F4853AF5
:101C7000910508F07CC08130910509F475C008F425
:101C8000E8C0049708F0E8C0E4C08F3B910508F075
:101C9000E0C0C85AD0E0CC0FDD1FC65BDE4F099014
:101CA000D881C02DCE019464D8C0811540E294073C
:101CB00058F4811551E0950708F0CEC08D3E91058E
:101CC00008F4C7C09065C9C0C11580E4D80708F4FE
:101CD000C0C0DF70CE01906AC0C0811525E59207B3
:101CE000A8F4811534E5930708F095C0811543E504
:101CF000940708F07BC0811552E5950708F061C094
:101D0000D82FCC27CE01816F906AA7C0C11589E575
:101D1000D807A0F4C11528E5D20708F082C0C11584
:101D200036E5D30708F095C08C2F0E94DC0F8F7129
:101D300090E0D82FCC27CE0190628FC0C1154AE524
:101D4000D40708F474C0CE0190568115904208F073
:101D500080C08D2F8F710E94DC0FDD27D0628F71C4
:101D6000AE01582BCA0179C081E090E076C0C55A17
:101D7000D0E0C858DE4F8881C82FD0E0CE019064F3
:101D80006CC074E0969587957A95E1F7282F2370BB
:101D90003C2F337081E090E002C0880F991F3A9584
:101DA000E2F79C68AC01522B9A019C2F9F7096958C
:101DB000969550E2959FE0011124C9018C2B9D2B33
:101DC0004CC08370992721E030E002C0220F331FFE
:101DD0008A95E2F79C2F9695969580E2989FE00170
:101DE0001124C22BD32BCE019C6837C08370992756
:101DF00021E030E002C0220F331F8A95E2F79C2FCA
:101E00009695969540E2949FE0011124C22BD32B26
:101E1000CE019A6822C0D82FCC27CE01846F906A59
:101E20001CC0DC2FCC27CE01806F906A16C08C2F8F
:101E30008F700E94DC0F94E0D695C7959A95E1F7D4
:101E4000CF70D0E0DC2FCC27D0699E01282BC901B0
:101E500004C080E090E001C0CE01DF91CF910895F1
:101E60002FE0829FC0011124FC0125E0729FE00D4C
:101E7000F11D1124E60FF11DEE0FFF1FE852FF4F79
:101E80008591949108950E94300F0E941E0E08952E
:101E90008238910569F1B0F48133910509F46DC080
:101EA00048F48932910509F463C08A32910509F436
:101EB00069C008958533910509F455C089339105AA
:101EC000B9F00895833E910569F138F4803E91059B
:101ED000B1F0823E910509F10895863E9105A9F180
:101EE000873E9105B9F1843E910509F064C023C095
:101EF00020911B0220FD4FC021FD4DC0089580910F
:101F00001B0280FD44C080911C0280FF44C0809170
:101F10001B0284FD42C083EE4DC080911B0282FFF4
:101F200038C0F5CF80911B0282FD33C080911C0226
:101F300080FD31C0ECCF80911C0281FF32C08091C6
:101F40001B0284FD2AC087EE35C080911B0283FFEF
:101F500026C0F5CF80911B0283FD21C080911C0219
:101F600081FD1FC0ECCF80911B0285FD1CC01DC0F0
:101F700080911B0285FD19C016C080911B0286FD51
:101F800016C017C080911B0286FD13C010C089E3E4
:101F900011C082EE0FC080EE0DC080E00BC086EE57
:101FA00009C084EE07C089E205C085E303C08AE268
:101FB00001C081E390E0089590911B0292FF0DC053
:101FC000282F2871283019F4877F846006C0282FB5
:101FD0002471243011F48B7F886093FF0DC0282F6B
:101FE0002871283119F4877E846106C0282F247156
:101FF000243111F48B7E886120911C0220FF0DC0DA
:10200000382F3871383019F4877F816006C0382F37
:102010003171313011F48E7F886021FF0DC0282F7F
:102020002871283119F4877E816106C0282F21711B
:10203000213111F48E7E886194FD877E089580E0C1
:1020400008950C94980C0E941E118FE39CE901974F
:10205000F1F700C000000E941E1180E00E945D1098
:1020600080FF04C00E9421100C94081808950C945D
:1020700023100E949E0C811102C00E94460D0E94F6
:10208000A90C8093F1010E94B10C90931C028093E3
:102090001B020E9437100E94AD0C682F70E080E098
:1020A00090E00E94B8066091920170919301809136
:1020B0009401909195010C94F006E82FF0E0E05E19
:1020C000FD4F80810895089580EA8A95F1F708957B
:1020D00000C008950C94641008950C946C100C9436
:1020E0006D100C946C100C947110F894E82FE2951C
:1020F000EF70F0E031A1282F2F7081E090E001C057
:10210000880F2A95EAF7982F9095932391A392A18F
:10211000892B82A378940895CF93DF9384EF0E9454
:10212000751085EF0E94751086EF0E947510CBE741
:10213000D1E089918F3F11F00E94751081E0C03885
:10214000D807B9F7DF91CF910895CF92DF92EF9240
:10215000FF920F931F93CF93DF938C01C62FD0E094
:10216000CE0180589E4F7C01FC0190819F3F09F475
:1021700047C0D62EF894E92FE295EF70F0E081A1E8
:102180009F7021E030E001C0220F9A95EAF7822B80
:1021900081A382A12095282322A378940E9468100D
:1021A000EBE7F1E040E851E031E0C12C21912F3F15
:1021B00089F0A22FA295AF70B0E090968C9190E03C
:1021C0002F7002C0959587952A95E2F780FD02C091
:1021D000832F01C080E0C82A330F4E175F0731F705
:1021E000F70180818F3F11F00E94751061E0C110EE
:1021F00001C060E08D2D0E946A10C00FD11FC882FF
:10220000DF91CF911F910F91FF90EF90DF90CF90D2
:1022100008950E948C1083E0E0E2F2E0DF01982F45
:102220001D929A95E9F7EDE1F2E0DF011D928A95A2
:10223000E9F783E00E9461110C94AA011F93CF93E8
:10224000DF9300D01F92CDB7DEB719821A821B82AE
:1022500060E0CE0101960E94A51061E0CE010196DA
:102260000E94A51062E0CE0101960E94A51043E0F5
:1022700050E0BE016F5F7F4F8DE192E00E94261F0C
:1022800011E0009709F410E0892B49F089819A81C7
:10229000AB8180931D0290931E02A0931F02212FF9
:1022A00043E060E272E08DE192E00E9462110E94E0
:1022B000AC01812F0F900F900F90DF91CF911F9164
:1022C00008950895FF920F931F93CF93DF938C018E
:1022D000F62ED72FC42F222349F081E08093F401FA
:1022E0000E94BB179093F3018093F2018091F40157
:1022F0008823C1F08091F2019091F3010E94D317DD
:10230000059780F0EF2DFD2FD8014C2F50E0CD0127
:10231000801B910B841795071CF48D918193F7CF47
:102320001092F401DF91CF911F910F91FF900895CA
:102330000E94BE190E948A0D0C94CA190E94CE19DF
:102340000E94180E0C94E8190E9459170E94A519B2
:102350000E94780D0E9498110E949E110E94820D89
:10236000FBCF8091FB0180FF06C06091090170E006
:10237000660F771F26C081FF04C06091090184E0C9
:1023800005C082FF07C06091090188E0689FB00125
:10239000112417C09091FA019923D1F0609108019E
:1023A000961788F72091090188E0289F9001112451
:1023B000929FA001939F500D112470E0CA010E94CA
:1023C000F81E6038710540F46115710519F406C0F6
:1023D00068E070E0862F08958FE7089581E0089502
:1023E0008091FB0180FF08C06091050170E0759548
:1023F00067957595679521C081FF06C060910501BD
:1024000070E07595679519C082FF04C06091050161
:1024100070E010C09091F901992399F06091040146
:102420009617A0F780910501899FC001112470E0E3
:102430000E94F81E6038710540F46115710519F4A9
:1024400006C061E070E0862F08958FE7089581E06F
:1024500008958D3E21F40E94B111819504C08E3EF5
:1024600029F40E94B1118093FF0108958F3E21F459
:102470000E94B111819504C0803F29F40E94B111DE
:102480008093FE010895893F19F40E94F01105C060
:102490008A3F31F40E94F0118195809300020895E3
:1024A0008B3F21F40E94F011819504C08C3F29F4E8
:1024B0000E94F0118093010208959FE0980F9830D8
:1024C00078F421E030E0A90102C0440F551F9A952D
:1024D000E2F7CA019091FD01892B8093FD010895D7
:1024E0008D3F21F48091FB0181600BC08E3F21F470
:1024F0008091FB01826005C08F3F29F48091FB0130
:1025000084608093FB0108958D3E39F49091FF0122
:1025100097FF35C01092FF0159C08E3E29F490916B
:10252000FF011916BCF32BC09091FE018F3E29F4D8
:1025300097FF25C01092FE0149C0803F19F419167B
:10254000CCF31DC090910002893F29F41916BCF408
:10255000109200023BC08A3F19F497FF10C0F8CFD9
:102560008B3F39F49091010297FF09C0109201024C
:102570002DC08C3F21F4909101021916BCF39FE00D
:10258000980F983080F421E030E0A90102C0440F98
:10259000551F9A95E2F7CA0180959091FD01892314
:1025A0008093FD0113C08D3F21F48091FB018E7F4C
:1025B0000BC08E3F21F48091FB018D7F05C08F3FC2
:1025C00029F48091FB018B7F8093FB018091FE01B8
:1025D000811106C08091FF01811102C01092FA01A1
:1025E00080910002811106C080910102811102C018
:1025F0001092F90108950E94BB172091FE0121114C
:1026000004C02091FF01222321F09093F8018093D0
:10261000F70120910002211104C020910102222320
:1026200021F09093F6018093F5018CEF91E00C94EA
:102630009916EF92FF920F931F93CF93DF9300D0E1
:1026400000D000D0CDB7DEB786E0ECEFF1E0DE01E0
:10265000119601900D928A95E1F7E090FE01F090BD
:10266000FF0100910002109101021092FE011092F0
:10267000FF011092000210920102E11003C0FF203E
:1026800009F45DC08091F7019091F8010E94D31781
:10269000AC019091FA01992339F020910A0130E0C0
:1026A0002417350758F04BC020910B018AE0289F72
:1026B000900111242417350718F041C09F3F19F0ED
:1026C0009F5F9093FA01EE2061F00E94B1111E14F9
:1026D00014F09FEF01C091E0989F902D11249093EA
:1026E000FE01FF2061F00E94B1111F1414F09FEF52
:1026F00001C091E0989F902D11249093FF0130919B
:10270000FE013323E1F02091FF012223C1F045EBCC
:102710003403C0011124992319F09093FE0103C0E2
:1027200081E08093FE0135EB2303C001112499233E
:1027300019F09093FF0103C081E08093FF01011124
:1027400003C0112309F45DC08091F5019091F60159
:102750000E94D317AC019091F901992339F020918F
:10276000060130E02417350758F04BC020910701CF
:102770008AE0289F900111242417350718F041C0E2
:102780009F3F19F09F5F9093F901002361F00E9431
:10279000F011101614F09FEF01C091E0989F902D5A
:1027A000112490930002112361F00E94F011111680
:1027B00014F09FEF01C091E0989F902D1124909309
:1027C0000102309100023323E1F020910102222323
:1027D000C1F045EB3403C0011124992319F0909303
:1027E000000203C081E08093000235EB2303C001A7
:1027F0001124992319F09093010203C081E0809382
:1028000001028091FE0181110BC08091FF018111B5
:1028100007C080910002811103C0809101028111E3
:102820000E94FB12EB82FC820D831E8386E0FE0178
:102830003196ACEFB1E001900D928A95E1F72696C2
:102840000FB6F894DEBF0FBECDBFDF91CF911F91C1
:102850000F91FF90EF900895ECEFF1E086E0DF013B
:102860001D928A95E9F71092FA011092F9011092DF
:10287000FB010895CF93DF93EC01FB018281882354
:1028800009F43CC1C430FDE5DF0760F4CB3F9CE5B3
:10289000D90788F49E0122503C452431310508F0C7
:1028A0002EC109C0C236EDE5DE0729F0C63AFDE5C6
:1028B000DF0709F024C10E94B10C90931C028093A1
:1028C0001B02C1318CE5D80709F4C6C008F042C02C
:1028D000C930ECE5DE0709F49BC000F5C5308CE596
:1028E000D80709F485C078F4C330ECE5DE0709F4B5
:1028F00078C008F07AC0C230DC4509F0F5C080919C
:102900001B028160EFC0C7309CE5D90709F478C08D
:1029100008F07AC080911B028061E4C0CD30FCE5F4
:10292000DF0709F487C058F4CB309CE5D90709F4D8
:1029300079C008F07BC080911B0288606FC0CF30E7
:10294000FCE5DF0709F480C008F082C080911B021B
:10295000877FC8C0CE3F9CE5D90709F471C000F558
:10296000C531FCE5DF0709F485C068F4C3319CE597
:10297000D90709F475C008F095C00E9460068091DF
:102980001B028F77AFC0CC3FFCE5DF07A9F108F051
:1029900054C0CB3FDC4509F0A7C080911C0240C069
:1029A000C230EDE5DE0709F489C058F4C1158DE5A4
:1029B000D80709F45AC008F069C080911C028260EF
:1029C0002FC0C236EDE5DE0709F47CC0C63AFDE54E
:1029D000DF0709F481C0C330DD4509F085C080E020
:1029E0006EC080911B0282607DC080911B0216C068
:1029F00080911B02886076C080911C0282604FC06B
:102A000080911B0280626EC080911B0280646AC04C
:102A10000E94600680911B02806864C0846062C06E
:102A200081603DC080911B028E7F5CC080911B0243
:102A30008D7F58C080911B0216C080911C0218C067
:102A400080911C028D7F2BC080911B028F7E4AC01B
:102A500080911B028F7D46C080911B028F7B42C0FC
:102A600080911B02877F8B7F3DC080911C028D7FF0
:102A70008E7F15C080911B0282FB222720F991E0F6
:102A8000922790FB82F990FB83F92CC080911C0265
:102A9000982F909591708E7F892B90FB81F9809370
:102AA0001C0222C00E94600680911B0287FB222725
:102AB00020F991E0922790FB87F914C081E00E94F1
:102AC000480D12C080911B0284FB222720F991E05F
:102AD000922790FB84F906C080911B02982F909555
:102AE00090FB80F980931B0280911B0290911C0245
:102AF0000E94C20C0E94600680E001C081E0DF916C
:102B0000CF910895CF93DF9386319C4541F5EB013A
:102B10000E94B50B982F8A81209102013091030108
:102B2000882379F09A7A81E009F480E080930202A8
:102B3000911102C069E201C065E3C9010E94151745
:102B40000AC080910202811102C069E201C065E3FE
:102B5000C9010E9417170E94F70B80E001C081E0B5
:102B6000DF91CF9108950F931F93CF93DF93C42FDD
:102B7000D22FFC0182818823C9F0409305020E9474
:102B8000BB17909304028093030280E28C0F88307D
:102B900008F057C0C77081E001C0880FCA95EAF7F6
:102BA000DF91CF911F910F910C94BD03809105028D
:102BB000481330C080910302909104020E94D31701
:102BC000883C910538F510E21D0FCD17B9F080E271
:102BD0008C0F883040F4C77081E001C0880FCA951F
:102BE000EAF70E94C403183028F581E09D2F977002
:102BF00001C0880F9A95EAF70E94BD03802F0E94BA
:102C0000B4031830F0F4D77081E001C0880FDA9572
:102C1000EAF70AC080E28C0F883098F4C77081E030
:102C200001C0880FCA95EAF7DF91CF911F910F91EC
:102C30000C94C403802FDF91CF911F910F910C94BE
:102C4000B403DF91CF911F910F9108950F939C01D1
:102C5000CB01243F4CE5340731F188F4293DFCE5F4
:102C60003F07D9F02A3D4CE5340779F1283D3C4532
:102C7000A9F506E221EE41EE68ED7CE52BC0263F8A
:102C8000FCE53F07E1F0A8F0273F3C4539F507E2B6
:102C900025EE46EE67EF7CE51DC007E225EE45EE2A
:102CA00069ED7CE517C006E221EE40EE64EF7CE5BD
:102CB00011C007E225EE44EE65EF7CE50BC006E2AD
:102CC00021EE42EE66EF7CE505C008E221E045EE2C
:102CD0006AED7CE50E94B31580E008C0FC018281AA
:102CE000882319F01092050201C081E00F91089528
:102CF0009093850180938401089590930B028093B3
:102D00000A020895E0910A02F0910B02309721F037
:102D10000190F081E02D099480E00895E0910A028D
:102D2000F0910B02309721F00280F381E02D09949D
:102D30000895E0910A02F0910B02309739F022E0F9
:102D4000DC012C930480F581E02D099408952091F5
:102D50000802309109022817390771F0909309028F
:102D600080930802E0910A02F0910B02309721F063
:102D70000680F781E02D0994089520910602309194
:102D800007022817390771F0909307028093060213
:102D9000E0910A02F0910B02309721F00084F18556
:102DA000E02D09940895FC01329697E080E091505F
:102DB00029F021912223D9F38F5FF9CF089566235B
:102DC00049F0FC01329608962191621729F0E81724
:102DD000F907D1F780E0089581E008959C01FC0196
:102DE00032969FEF80E04191461789F09F3F19F49A
:102DF000411101C0982F8F5F8630A9F79F3F39F0AE
:102E0000F901E90FF11D97FDFA9562830895089580
:102E10009C012A5F3F4FFC014281461301C0128290
:102E2000019682179307B9F708950C94EE160C9447
:102E30000817029626E0FC0111922A95E9F70895F9
:102E400008950C94201783E080930C020C942117B2
:102E5000811102C081E001C082E080930C020C94D9
:102E600021170C94281781E080930C020C942117F1
:102E70000C94331708950C943A170C943B170C9448
:102E80003A170C943A170C943A17CF930E944117B3
:102E90000E941E110E943F17C0E08C2F0E945D10FF
:102EA000811104C0CF5FC330C1F701C081E0CF9171
:102EB000089508951F920F920FB60F9211248F93C9
:102EC0009F93AF93BF9380910D02811113C08091A6
:102ED000230290912402A0912502B09126024196EE
:102EE000A11DB11D8093230290932402A09325027B
:102EF000B0932602BF91AF919F918F910F900FBE1B
:102F00000F901F90189580912B02843031F10E9410
:102F1000100210920D0220E488E190E00FB6F894C0
:102F2000A895809360000FBE2093600083B7817FD7
:102F3000846083BF83B7816083BF7894889583B7AB
:102F40008E7F83BF0FB6F894A8958091600088614A
:102F500080936000109260000FBE08950E9460068A
:102F60000C94140282E084BD93E095BD9AEF97BD66
:102F700080936E0008952FB7F8948091230290916A
:102F80002402A0912502B09126022FBF08952FB7E9
:102F9000F89460912302709124028091250290910F
:102FA00026022FBF08959C014FB7F8948091230209
:102FB00090912402A0912502B09126024FBF821B5E
:102FC000930B089578941F920F920FB60F921124CD
:102FD0008F939F93AF93BF9380912302909124028C
:102FE000A0912502B09126020196A11DB11D8093EA
:102FF000230290932402A0932502B0932602BF914E
:10300000AF919F918F910F900FBE0F901F901895C9
:1030100081E08093E00080E28093D8001092C900A4
:103020008FE19EE40197F1F700C0000087E090EB8C
:10303000DC018093340290933502A0933602B09362
:1030400037029CE088E10FB6F894A8958093600061
:103050000FBE90936000FFCF8091190208950895EC
:1030600022E02093E9002FEF3091E800215035FD58
:1030700006C035ED3A95F1F700002111F5CF20910A
:10308000E80025FF0BC040E050E066E070E00E94E1
:103090005A1A8091E8008E778093E8000895CF93C4
:1030A000DF9321E02093E9002FEF3091E8002150D9
:1030B00035FD06C035ED3A95F1F700002111F5CF49
:1030C0002091E80025FF14C0EC0140E050E068E0EA
:1030D00070E00E945A1A8091E8008E778093E80091
:1030E00088E0FE01A1E1B2E001900D928A95E1F73E
:1030F000DF91CF91089580930E0270931002609338
:103100000F0280912B02843001F582E08093E90068
:103110008FEF9091E800815095FD06C095ED9A954E
:10312000F1F700008111F5CF8091E80085FF0DC017
:1031300040E050E063E070E08EE092E00E945A1AB6
:103140008091E8008E778093E8000895BC0184E0C8
:103150000C947B18BC0183E00C947B1880912A02AC
:10316000811109C00E94EB1B0E94481C8091E20063
:1031700084608093E200089510922A0208950C94CE
:1031800038176091270281E0611101C080E00C9442
:10319000231790912B0281E0943009F080E0609138
:1031A00027020C94281742E061EC81E00E94641B26
:1031B00042E261EC82E00E94641B90912B0281E06C
:1031C000943009F080E0609127020C9431178091CF
:1031D0002D02833009F461C030F4813071F0823007
:1031E00009F49AC008958A3009F486C08B3009F436
:1031F0006CC0893009F0A8C020C080912C02813AAF
:1032000009F0A2C08091E800877F8093E800809158
:10321000300290913102892B21F468E081E192E043
:1032200003C060E080E090E070E00E94A51A809109
:10323000E8008B778093E800089580912C0281321A
:1032400009F082C08091300290913102029708F01B
:103250007BC08091E800877F8093E8008091E80040
:1032600082FD05C080912B028111F8CF6DC02091A5
:10327000F3008091F20090E0922B029731F480915C
:10328000F100813011F0863021F48091F1008093BB
:1032900019028091E8008B7753C080912C02813A0B
:1032A00009F052C08091300290913102892B09F0CF
:1032B0004BC08091E800877F8093E8008091E80010
:1032C00080FFFCCF8091180136C080912C028132A2
:1032D000D9F58091300290913102892BA9F5809126
:1032E000E800877F8093E8000E94991B80912E025E
:1032F000809318010C94600680912C02813221F594
:103300008091E800877F8093E8000E94991B80915C
:103310002F0280931A02089580912C02813AA1F421
:103320008091E800877F8093E8008091E80080FF2B
:10333000FCCF80911A028093F1008091E8008E7793
:103340008093E8000C94991B089584B7877F84BF0D
:103350000FB6F894A8958091600088618093600012
:10336000109260000FBE90E080E80FB6F894809352
:103370006100909361000FBE0C9433170E94EB1B09
:103380000E94481CE2EEF0E08081846080837894A3
:103390000C94DD1E8CE091E00C947D1680912B0244
:1033A0008530A9F480912B02853079F40E9483172F
:1033B000809129028823B1F30E944517882391F355
:1033C0000E94441A0E946006EDCF0C94AE17089537
:1033D00008950C94EB19292F332723303105C9F0B8
:1033E00060F42130310581F02230310509F044C00C
:1033F0008BE390E024E331E043C021323105E1F07A
:103400002232310549F138C082E190E02FE631E007
:1034100037C099278130910549F028F0029761F56E
:10342000E6EFF0E005C0E0E3F1E002C0E6E1F1E044
:10343000849190E09F0124C06115710541F06130D5
:103440007105D1F489E090E02FE531E019C089E001
:1034500090E026E431E014C06115710541F061305F
:10346000710551F48BE790E021E831E009C080E478
:1034700090E02CEF31E004C080E090E020E030E00C
:10348000FA0131832083089580E189BD82E189BDFD
:1034900009B400FEFDCF8091D8008F7D8093D800C5
:1034A0008091E00082608093E0008091E00081FDE7
:1034B000FCCF0895CF92DF92EF92FF920F931F936C
:1034C000CF93DF93EC018B017A010E94B81B81112D
:1034D00033C0E114F10439F0F70180819181081BB8
:1034E000190BC80FD91FC12CD12C0115110519F1C9
:1034F0008091E80085FD16C08091E8008E7780936A
:10350000E800E114F10449F0F70180819181C80ECF
:10351000D91ED182C08285E00FC00E94B81B8823CB
:1035200021F30AC089918093F10001501109FFEF46
:10353000CF1ADF0ADACF80E0DF91CF911F910F9190
:10354000FF90EF90DF90CF9008952091320230915C
:1035500033022617370748F06115710539F42091B9
:10356000E8002E772093E80001C0B901FC0120E0BB
:103570006115710579F180912B028823F1F1853075
:10358000F1F18091E80083FD3CC08091E80082FD6C
:103590002EC08091E80080FFEBCF2091F300809156
:1035A000F20090E0922B6115710551F08830910581
:1035B00038F421912093F100615071090196F3CF05
:1035C00021E0089709F020E08091E8008E77809351
:1035D000E800CECF2111CFCF0AC080912B028823E3
:1035E00061F0853061F08091E80083FD0AC0809130
:1035F000E80082FFF2CF80E0089582E0089583E042
:10360000089581E008952091320230913302261707
:10361000370748F06115710539F42091E8002E77DD
:103620002093E80001C0B901FC0120E0611571059B
:1036300091F180912B02882309F440C0853009F470
:103640003FC08091E80083FD3DC08091E80082FD8D
:103650002FC08091E80080FFE9CF2091F300809196
:10366000F20090E0922B6115710559F088309105B8
:1036700040F424912093F100319661507109019634
:10368000F2CF21E0089709F020E08091E8008E77E2
:103690008093E800CBCF2111CCCF0AC080912B02C0
:1036A000882361F0853061F08091E80083FD0AC0D5
:1036B0008091E80082FFF2CF80E0089582E00895D3
:1036C00083E0089581E00895982F973068F59093EE
:1036D000E900981739F07091EC002091ED005091BD
:1036E000F00003C0242F762F50E021FD02C09F5F21
:1036F000ECCF3091EB003E7F3093EB003091ED004A
:103700003D7F3093ED003091EB0031603093EB0062
:103710007093EC002093ED005093F0002091EE00A8
:1037200027FDE5CF80E008958F708093E90081E068
:10373000089580912C0287FF11C08091E80082FDDE
:1037400005C080912B028111F8CF11C08091E80053
:103750008B770BC080912B02882349F08091E80081
:1037600080FFF8CF8091E8008E778093E80008957D
:103770002091E4003091E50095E64091EC00842F23
:10378000817040FF23C08091E80080FD1DC08091C2
:103790002B02882399F0853099F08091EB0085FD0C
:1037A00011C04091E4005091E5002417350729F33A
:1037B000915011F09A01E1CF84E0089582E00895DC
:1037C00083E0089581E0089580E008954091E80045
:1037D00042FFDDCF08950E94591C0E94611CE0EE5B
:1037E000F0E0808181608083E8EDF0E080818F7778
:1037F000808319BCA7EDB0E08C918E7F8C93808183
:103800008F7E808310922A0208950F931F93CF9387
:10381000DF930E94591C0E94611CC8EDD0E0888192
:103820008F77888388818068888388818F7D88836B
:1038300019BC10922B0210922702109229021092AA
:10384000280200EE10E0F80180818B7F8083888160
:103850008160888342E060E080E00E94641BE1EECA
:10386000F0E080818E7F8083E2EEF0E080818160F5
:103870008083808188608083F80180818E7F80834F
:10388000888180618883DF91CF911F910F91089586
:10389000E8EDF0E080818F7E8083E7EDF0E08081CD
:1038A0008160808384E082BF81E080932A020C944F
:1038B000051CE8EDF0E080818E7F80831092E200AD
:1038C00008951092DA001092E10008951F920F926D
:1038D0000FB60F9211242F933F934F935F936F93E3
:1038E0007F938F939F93AF93BF93EF93FF938091B9
:1038F000E10082FF0BC08091E20082FF07C080914F
:10390000E1008B7F8093E1000E94DC1E8091DA0051
:1039100080FF1FC08091D80080FF1BC08091DA001B
:103920008E7F8093DA008091D90080FF0DC080E106
:1039300089BD82E189BD09B400FEFDCF81E080939D
:103940002B020E94AE1805C019BC10922B020E94D7
:10395000BC188091E10080FF19C08091E20080FFD7
:1039600015C08091E2008E7F8093E2008091E2009A
:1039700080618093E2008091D80080628093D800BB
:1039800019BC85E080932B020E94C1188091E10050
:1039900084FF30C08091E20084FF2CC080E189BDAB
:1039A00082E189BD09B400FEFDCF8091D8008F7DF2
:1039B0008093D8008091E1008F7E8093E100809118
:1039C000E2008F7E8093E2008091E200816080932C
:1039D000E20080912702882311F084E007C08091E3
:1039E000E30087FD02C081E001C083E080932B02E9
:1039F0000E94C9188091E10083FF29C08091E200F4
:103A000083FF25C08091E100877F8093E10082E001
:103A100080932B02109227028091E1008E7F809389
:103A2000E1008091E2008E7F8093E2008091E200CD
:103A300080618093E20042E060E080E00E94641BCD
:103A40008091F00088608093F0000E94BF18FF9181
:103A5000EF91BF91AF919F918F917F916F915F9106
:103A60004F913F912F910F900FBE0F901F9018957F
:103A70001F920F920FB60F9211242F933F934F93E3
:103A80005F936F937F938F939F93AF93BF93CF93E6
:103A9000DF93EF93FF93C091E900CF708091EC002A
:103AA000D82FD17080FDD0E81092E9008091F0000D
:103AB000877F8093F00078940E947C1D1092E9002B
:103AC0008091F00088608093F000CD2BCF70C09380
:103AD000E900FF91EF91DF91CF91BF91AF919F915D
:103AE0008F917F916F915F914F913F912F910F90A7
:103AF0000FBE0F901F9018951F93CF93DF93CDB7F4
:103B0000DEB7AA970FB6F894DEBF0FBECDBFECE2CA
:103B1000F2E08091F100819322E0E433F207C9F7EB
:103B20000E94E7188091E80083FF2EC180912C024B
:103B300090912D02492F50E04A30510508F024C1E0
:103B4000FA01EE59FF4F0C940C1F803821F0823897
:103B500009F01AC108C08091280290912902992386
:103B600089F082600FC0809130028F70873008F03A
:103B70000BC18093E9008091EB0085FB882780F9D9
:103B80001092E9009091E800977F9093E80080936D
:103B9000F1001092F100D1C0282F2D7F09F0F4C060
:103BA000882319F0823061F0EFC080912E028130BD
:103BB00009F0EAC0933009F080E0809329022EC01A
:103BC00080912E0281112AC0809130028F702FEFD8
:103BD000280F263008F0D8C08093E9002091EB0030
:103BE00020FF1CC0933021F48091EB00806214C050
:103BF0009091EB0090619093EB0021E030E0A901FF
:103C000002C0440F551F8A95E2F74093EA001092D4
:103C1000EA008091EB0088608093EB001092E9004D
:103C20008091E800877F8093E8000E94991BACC0D8
:103C30008111AAC010912E021F778091E300807835
:103C4000812B8093E3008091E800877F8093E800D8
:103C50000E94991B8091E80080FFFCCF8091E300D7
:103C600080688093E300111102C082E001C083E00C
:103C700080932B0289C08058823008F085C08091E3
:103C80002E0290912F028C3D53E0950779F583E049
:103C90008A838AE289834FB7F894DE01139620E085
:103CA0003EE051E2E32FF0E050935700E49120FF13
:103CB00003C0E295EF703F5FEF708E2F90E0EA3027
:103CC00010F0C79601C0C0968D939D932F5F24314D
:103CD00049F74FBF8091E800877F8093E8006AE250
:103CE00070E0CE0101960E94A51A16C060913002C4
:103CF00070913102AE014F5F5F4F0E94E919BC0124
:103D0000892B09F441C09091E800977F9093E800D7
:103D100089819A810E94031B8091E8008B778093B0
:103D2000E80032C0803881F58091E800877F809379
:103D3000E800809127028093F1008091E8008E775F
:103D400072CF811121C080912E0290912F0299276C
:103D50000297D4F48091E800877F8093E8008091F7
:103D60002E02809327020E94991B809127028111C5
:103D700006C08091E30087FD02C081E001C084E0BD
:103D800080932B020E94D3188091E80083FF0AC021
:103D90008091E800877F8093E8008091EB0080624B
:103DA0008093EB00AA960FB6F894DEBF0FBECDBF8E
:103DB000DF91CF911F9108950895CF9380912B02A9
:103DC0008823A1F0C091E900CF709091EC00892F79
:103DD000817090FD80E8C82B1092E9008091E80086
:103DE00083FD0E947C1DCF70C093E900CF910895A0
:103DF00097FB072E16F4009407D077FD09D00E9498
:103E0000121F07FC05D03EF4909581959F4F0895B1
:103E1000709561957F4F0895EE0FFF1F0590F49107
:103E2000E02D0994AA1BBB1B51E107C0AA1FBB1FB1
:103E3000A617B70710F0A61BB70B881F991F5A9536
:103E4000A9F780959095BC01CD010895FB01DC0197
:103E500004C08D910190801921F441505040C8F761
:103E6000881B990B0895F999FECF92BD81BDF89AF0
:103E7000992780B50895A8E1B0E042E050E00C94A5
:103E8000671F262FF999FECF92BD81BDF89A019741
:103E900000B4021639F01FBA20BD0FB6F894FA9A92
:103EA000F99A0FBE08950396272F0E94421F0E9481
:103EB000411F252F0E94421F242F0C94421F019660
:103EC000272F0E94421F0C94411FDC01CB01FC01F3
:103ED000F999FECF06C0F2BDE1BDF89A319600B463
:0E3EE0000D9241505040B8F70895F894FFCF6E
:103EEE00C800DC01280850011E0A14012C184F18B6
:103EFE003018AA18A6182F1801E200E900EA00B53A
:103F0E0000B600B700CD008301CC008A0192019467
:103F1E00012102230224022502260227022A02B3CD
:103F2E0000B4006F007000818283E200E900EA00B5
:103F3E00B500B600B700CD008301CC008A01920116
:103F4E0094012102230224022502260227022A02BC
:103F5E00B300B4006F007000818283F731333236C4
:043F6E00F4F5F60070
:00000001FF
